:10000000A4C1BCC1BBC1BAC1B9C1B8C1B7C1B6C135
:10001000B5C1B4C1B3C1B2C1B1C1B0C1AFC1AEC14C
:10002000ADC1ACC1ABC1A4C1BCC1BBC1BAC1B9C136
:10003000B8C1B7C1B6C1B5C1B4C1B3C1B2C1B1C114
:10004000B0C1AFC1AEC1ADC1ACC1ABC1FFFF1124E6
:100050001FBECFEDCDBF10E0A0E6B0E0E6E4F6E0D5
:1000600002C005900D92A036B107D9F710E0A0E6C6
:10007000B0E001C01D92A036B107E1F713D163C112
:1000800041CE27E030E090E0482F50E0D898BA0108
:10009000022E02C0759567950A94E2F760FF02C0D0
:1000A000919A01C091980000000000000000D89AC9
:1000B000990FC999916000000000000000002150D4
:1000C00030408FEF2F3F380709F7D898892F0895D0
:1000D000CF93DF93CDB7DEB7C350CDBF2B834A8319
:1000E0006983CFDF6981862FCCDF4A81842FC9DF06
:1000F0002B81822FC6DFCD5FCDBFDF91CF910895D9
:10010000CF938CEABEDF83E5BCDF80E0BADFC82F87
:1001100080E0B7DF81E0C33509F080E0CF9108953A
:100120008CEA60E840E020E0D3DF0895982F242F88
:10013000662311F088E401C080E460E0492FC8DF45
:100140000895682F62956370482F50E084E0440F53
:10015000551F8A95E1F78CE420E0BADF83EC99E043
:100160000197F1F700C000000895CF92DF92EF925F
:10017000FF920F931F93CF93DF936B01E3ECF9E0B2
:100180003197F1F700C000007C01C0E0D0E000E052
:1001900010E01EC0F70144918C2F60E0C7DFF7012B
:1001A000319644918C2F61E0C1DFCF5FC03131F0D7
:1001B00098012E5F3F4F2C153D0520F08D2FC1DF9C
:1001C000DF5FC0E00E5F1F4F82E090E0E80EF91E97
:1001D0000C151D05F8F2DF91CF911F910F91FF9043
:1001E000EF90DF90CF9008958F929F92AF92BF9241
:1001F000CF92DF92EF92FF920F931F93CF93DF93F3
:100200005C014B0183EC99E00197F1F700C000001D
:1002100000E010E0FF24CC24DD2401C001E0C0E0B8
:10022000D0E006C0E60100E003C0E60100E010E017
:10023000F501EC0FFD1F4491FE013196EA0DFB1D07
:10024000E4904F3F51F49FEFE91639F4002331F366
:1002500092E0C92ED12CCC0EDD1E812F60E066DF2E
:10026000812F61E04E2D62DF22961F5F103129F051
:10027000C815D905E8F20023A9F68F2D62DFF394A3
:10028000C815D905A0F2013081F2DF91CF911F91FD
:100290000F91FF90EF90DF90CF90BF90AF909F9025
:1002A0008F900895C69A8FE996E8A1E0815090401A
:1002B000A040E1F700C0000080E0B699FDCF8F5F5D
:1002C0008A30D8F3C698D09A899A889A8FE39DE0AD
:1002D000A3E081509040A040E1F700C0000010DF93
:1002E0001FDF86E290E064E273E07EDFD0988998B9
:1002F00088988A9A929A8FE996E8A1E08150904076
:10030000A040E1F700C0000092988A988FE996E833
:10031000A1E081509040A040E1F700C000008FE9CB
:1003200096E8A1E081509040A040E1F700C00000B5
:10033000D998D19AA7EAB1E61197F1F700C0000069
:10034000D1980000FECFF894FFCF11241FBECFED4F
:10035000CDBF10E0A0E6B0E0E6E4F6E002C0059014
:100360000D92A036B107D9F710E0A0E6B0E001C0C9
:100370001D92A036B107E1F713D163C141CE27E04A
:1003800030E090E0482F50E0D898BA01022E02C029
:10039000759567950A94E2F760FF02C0919A01C0D3
:1003A00091980000000000000000D89A990FC999A8
:1003B00091600000000000000000215030408FEFED
:1003C0002F3F380709F7D898892F0895CF93DF93E7
:1003D000CDB7DEB7C350CDBF2B834A836983CFDF50
:1003E0006981862FCCDF4A81842FC9DF2B81822F40
:1003F000C6DFCD5FCDBFDF91CF910895CF938CEA5B
:10040000BEDF83E5BCDF80E0BADFC82F80E0B7DF66
:1004100081E0C33509F080E0CF9108958CEA60E86F
:1004200040E020E0D3DF0895982F242F662311F0B9
:1004300088E401C080E460E0492FC8DF0895682F98
:1004400062956370482F50E084E0440F551F8A95F1
:10045000E1F78CE420E0BADF83EC99E00197F1F753
:1004600000C000000895CF92DF92EF92FF920F93A9
:100470001F93CF93DF936B01E3ECF9E03197F1F732
:1004800000C000007C01C0E0D0E000E010E01EC031
:10049000F70144918C2F60E0C7DFF701319644915A
:1004A0008C2F61E0C1DFCF5FC03131F098012E5F4A
:1004B0003F4F2C153D0520F08D2FC1DFDF5FC0E0E1
:1004C0000E5F1F4F82E090E0E80EF91E0C151D052F
:1004D000F8F2DF91CF911F910F91FF90EF90DF9095
:1004E000CF9008958F929F92AF92BF92CF92DF925A
:1004F000EF92FF920F931F93CF93DF935C014B0119
:1005000083EC99E00197F1F700C0000000E010E0F3
:10051000FF24CC24DD2401C001E0C0E0D0E006C00F
:10052000E60100E003C0E60100E010E0F501EC0F99
:10053000FD1F4491FE013196EA0DFB1DE4904F3FF3
:1005400051F49FEFE91639F4002331F392E0C92EFC
:10055000D12CCC0EDD1E812F60E066DF812F61E0A3
:100560004E2D62DF22961F5F103129F0C815D90584
:10057000E8F20023A9F68F2D62DFF394C815D905A0
:10058000A0F2013081F2DF91CF911F910F91FF9086
:10059000EF90DF90CF90BF90AF909F908F90089595
:1005A000C69A8FE996E8A1E081509040A040E1F71B
:1005B00000C0000080E0B699FDCF8F5F8A30D8F38D
:1005C000C698D09A899A889A8FE39DE0A3E08150DB
:1005D0009040A040E1F700C0000010DF1FDF86E27E
:1005E00090E064E273E07EDFD098899888988A9AD8
:1005F000929A8FE996E8A1E081509040A040E1F7FF
:1006000000C0000092988A988FE996E8A1E0815096
:100610009040A040E1F700C000008FE996E8A1E01B
:1006200081509040A040E1F700C00000D998D19AD5
:10063000A7EAB1E61197F1F700C00000D1980000D9
:06064000FECFF894FFCF8D
:00000001FF
